:020000040000FA
:060000000219FD02031CC1
:03000B0002008D63
:03001300020535AE
:03001B0002009050
:03002B000202D1FD
:03005B0002054457
:030073000203097C
:100080000406080C10182030406080A0C0054032E3
:10009000C2AFC2A853E6EFC28E856B8BC0D0D2D35D
:1000A000C0E0C0F0C2CAA8CCA9CDD2CAD2AF758A6E
:1000B00000C3E8956CF8E9956DF9C3E913F9E81305
:1000C000F8E5666007C3E913F9E813F8E97025E875
:1000D000956E4020956E501CE582B410177C007B15
:1000E000007A007908900000A86AE5667004C3E809
:1000F00013F801FD900000D2A8D2AA61E7E0FDC389
:100100009CC39840EF98EB33FB0582E0FCC39DC392
:100110009840E198EB33FB0582E0FDC39CC3984017
:10012000D398EB33FB0582E0FCC39DC39840C59890
:10013000EB33FB0582E0FDC39CC39840B798EB33DB
:10014000FB0582E0FCC39DC39840A998EB33FB05F7
:1001500082E0FDC39CC398409B98EB33FB0582E093
:10016000FCC39DC398408D98EB33FB0582217890AA
:100170000000D2A8D2AA61E7E0FDC39CC39840EF7B
:1001800098EA33FA0582E0FCC39DC39840E198EAFF
:1001900033FA0582E0FDC39CC39840D398EA33FA52
:1001A0000582E0FCC39DC39840C598EA33FA0582F6
:1001B000E0FDC39CC39840B798EA33FA0582E0FC9F
:1001C000C39DC39840A998EA33FA0582E0FDC39C19
:1001D000C398409B98EA33FA0582E0FCC39DC3981C
:1001E000408D98EA33FA0582EBC46B6A54F0F9EA61
:1001F000C454F0C3996009900000D2A8D2AA61E764
:10020000EBF4C454F0F9EAF4C4540F49FAEBF4C423
:10021000540FFBC3EAF99460FAEB9400FB5020C33F
:10022000E97B007A0079006016C3135006F9C39584
:1002300052600AE9F5527553007900800205533087
:100240003A27C3EA94D0F8EB9407F9400BE8FAE9AF
:10025000FB203509D235415D303502C235203902E7
:10026000B235C3EA33FAEB33FBEB2B3B3BF9C3EB81
:1002700013FBEA13FAEA29FAEB3400FB30E3047AC1
:10028000FF7BFFE5255403601B202A18E55D33F949
:10029000EB7007C3E99A4002E9FAE53CC4332AFA55
:1002A000EB3400FBC3EA33C4540FF8EB33C454F00F
:1002B00048F87005EA60027801900000D2A8D2AA3E
:1002C000E5226002152281D4900000D2A8D2AA6152
:1002D000E7C0D0C0E0C2CF0541E5666009E56560D2
:1002E000057565006104756501E52360021523C38A
:1002F000E55460057555006104E5552401F5555038
:10030000037555FFD0E0D0D032C2AF53E67F75926F
:10031000FA7593FFC22053917FD2AF32C0E0E58AD5
:10032000303408856B8BF0A3D0E032D0E0C2AF53FD
:10033000E6EFC0D0C0E0C0F0D2D3D2AF5388EFA870
:100340008AA98CAA40308D010A758A00758C0075C7
:100350004000438810E566700AC3E833F8E933F9D2
:10036000EA33FA30331FE8C4540FFAE9C454F04AB0
:10037000FAC3132AFAC3E833F8E933F9E82AFAE9A9
:100380003406FB61D830320FC3E833E933FAE82A88
:10039000FAE93400FB61D8303115E875F056A4AAAB
:1003A000F0E975F056A42AFAC5F03400FB61D8C311
:1003B000EA13FAE913F9E813F8E875F056A4AAF07D
:1003C000E975F056A42AFAC5F03400C313FBEA130A
:1003D000FAC3EB13FBEA13FAC3EB94125009C3EA16
:1003E0009434EB940750160522E52270021522C3BF
:1003F000E52294325002A128755400A12BE5226019
:100400000215223036067C007D088117AC31AD32F2
:10041000303A04AC33AD34C3EA9CFAEB9DFB92084E
:10042000AE60AF61303A425007203509D235813590
:10043000303502C235303504AE62AF63203902B2C6
:1004400035C3EA33FAEB33FBA208500AEAF424017D
:10045000FAEBF43400FBC3EA9450FAEB9400FB503F
:100460001478007A007B008175A208500878007A21
:10047000007B0081D4E5255403601B202A18E55D2C
:1004800033F9EB7007C3E99A4002E9FAE53CC4335B
:100490002AFAEB3400FBEA8EF0A4F9AAF0EB8EF016
:1004A000A42AFAC5F03400FBC3EB13FDEA13F8C32A
:1004B000ED13FDE813F80FEF146004C3E833F8C33D
:1004C000E933EA33FAEB33FBDFEDEB30E30678FF99
:1004D0007AFF7B078854D230E86003755500C3E586
:1004E0005BFC955C4002AC5CC3EC95545008EC7529
:1004F000F008A4FAABF0EAF4F8EBF45407F9C3E817
:10050000941EFAE99400FB50047A007B0088568917
:10051000578A588B5975230AD0F0D0E0D0D053F7C2
:10052000DF43F74043E6103275230AD0F0D0E0D025
:10053000D043E61032C2AAD28EC2CA85CC6C85CD19
:100540006DD2CA32C2AFC0D0C0E0D2D3A8F9E55A4A
:1005500030E20AE5FA20E23520E132A165E5FA3021
:10056000E22B20E128C3E55713F8E55613F5E98897
:10057000EAC3E55913F8E55813F5FB88FC85575A8B
:1005800053F7BFD2A8303402D2AA53E6EF53F7DFB5
:10059000D0E0D0D0D2AF32790180147903801079C5
:1005A0000A800C791E80087964800479C8800078FC
:1005B00017E4D5E0FDD8FAD9F62278FF202828796B
:1005C000A1E76023E548601F74FF8548F084853FFC
:1005D000F030290375F005A4F8C5F0600278FFC378
:1005E000E8955D5002A85D885C22C3E54794A0E5CC
:1005F000489400E55C500314A1FB046002F55C2202
:1006000075E89022055EC3E55E9408405330EDF432
:10061000A8BDA9BE755E00E9FA79A0E76041EA705D
:1006200006E55F6018800CC3E8955F600EE55F50DB
:1006300005600A1480070460FA8002E55FF55FC375
:100640009569401B755BC0C394044013755B80C300
:100650009404400B755B40C394044003755B002217
:10066000E55B2410500274FFF55B22743279A68793
:10067000F0A4C5F0A2F733F55D227547007548F088
:1006800022C2AFC2CAA8CCA9CDAA4130CF010AD29A
:10069000CAD2AFC3EA13FAE913F9E813F8AB42ACD4
:1006A0004388428943C3E89BF8E99C20280A547F89
:1006B000F9302C02E19FC1F8AD448A44F9EA9D5417
:1006C0007FFA600678FF79FFC1DDAE45AF468B4506
:1006D0008C46A842A943C3E89EF8E99FF9C3E548C0
:1006E00013FBE54713FAE82AF547E93BF5485006BE
:1006F0007547FF7548FFE145AA47AB48AC47AD4891
:100700007E047F02C3EB9404400D1E1FC3EB9408CC
:1007100040052029021E1FC3ED13FDEC13FCDEF77C
:10072000C3EA9CFAEB9DFBEF6009C3E913F9E813F8
:10073000F8DFF7EA28FAEB39FB8A478B4850067B4B
:10074000FF8B478B48C3EB94025002D22C30280415
:100750007F03E1707892E6FFC3E53D948240110F7C
:10076000C3E53D94A040010FC3EF940640027F050E
:100770007E02E548C4540FF9E548C454F0F8E54753
:10078000C4540F28F8C3E89EFAE99400FB4009C35B
:10079000EA9401EB940050047A01E4FB0207EBAA0F
:1007A00047AB48EBC4FEEAC4540F4EFCC3EA9CFAC4
:1007B000EB9400FBC3E813C313F8EA28FAEB340008
:1007C000FB8A478B48C3EB94024002C22C7802EBB1
:1007D000C4FE7B00EAC4540F4EFAC3EA98FA4005FF
:1007E000C3940150027A017892E6FF302002E1EBD7
:1007F000854E92854F93D22043E680C3E49AF8E475
:100800009BF9C3E833F8E933F9302C03020880E898
:10081000FAE9FBD3E913FDE813FC884E894FC3EFD7
:1008200094036038EF20E00CE82CF8E93DF9ECFA8D
:10083000EDFB8013E828F8E939F9C3E82401F8E969
:100840003400F97AFF7BFFC3EF9403400F8A508B8B
:1008500051884A894B8C4C8D4D0208B5885089517E
:100860008A4A8B4B8C4C8D4D3028127550F0755147
:10087000FF754CF0754DFF754EF0754FFF0208B5D2
:10088000E8FAD3E813FC884EC3EF94036021EF200D
:10089000E007E82CF8ECFA01A0E8282401F87AFF38
:1008A000C3EF940340098A50884A8C4C0208B588EB
:1008B000508A4A8C4C30200201B5753A02D220434E
:1008C000E680E5255403602DA847A948C3E913F93C
:1008D000E813F8302804E92440F9C2AF53E67F75E5
:1008E0009100C3E498F594E499F595759104D220AC
:1008F00043E680D2AF22D221754900752000302B0B
:10090000037520402114D221754900752040302BF9
:100910000375200078017901202C20E5255403601F
:1009200002C2217914E548C313700104F8C394147A
:1009300040027814302804781B791BC3E833F8C3CD
:10094000E933F9202010E549600C302803D53A043A
:10095000D22221C711BD0549E59B5440B520022193
:10096000B130280908C3E899400118214320210A21
:1009700008C3E899400221142143C22153E67F7540
:100980009100302C117594007595F0759104D2206A
:1009900043E680020914E5487EFFC3334009C333B0
:1009A0004005C3334001FEC3E49E759400F59521D4
:1009B0008BC3E5399401500221143021022114D84F
:1009C0000221C52143C222C2AF53E67F7591008543
:1009D0005094855195759104854A92854B93D22008
:1009E00043E680D2AFE5255403600720290205398C
:1009F000801030220D202B0A20210715811581023D
:100A000014312278003021027801E53D75F007A409
:100A1000F9E5F028F5F0E9A2F013A2F113A2F21320
:100A2000F53DC394785003753D78C3E53D953E4050
:100A30000653F28F75D5FF3020024137854C9285E1
:100A40004D93D22043E68022203817C2AF53F2DF05
:100A5000C29643F24075D5EF43F210D2AF759F5363
:100A6000616CC2AF53F2DFC29443F21075D5BF433D
:100A7000F240D2AF759F53616C203817C2AF53F26A
:100A8000EF75D5DF43F220C29643F240D2AF759F97
:100A900063616CC2AF53F2BF75D5DF43F220C294DD
:100AA00043F210D2AF759F23616C203817C2AF5349
:100AB000F2BFC29443F21075D5DF43F220D2AF7576
:100AC0009F23616CC2AF53F2EFC29643F24075D5DB
:100AD000DF43F220D2AF759F63616C203817C2AF3D
:100AE00053F2DF75D5BF43F240C29443F210D2AF48
:100AF000759F538077C2AF53F2DF75D5EF43F21085
:100B0000C29643F240D2AF759F538060203817C21F
:100B1000AF53F2EFC29543F22075D5BF43F240D2F6
:100B2000AF759F638046C2AF53F2BFC29543F220B8
:100B300075D5EF43F210D2AF759F23802F20381761
:100B4000C2AF53F2BF75D5EF43F210C29543F22006
:100B5000D2AF759F238015C2AF53F2EF75D5BF4357
:100B6000F240C29543F220D2AF759F63227A147B84
:100B70007880127A107B8C800C7A0D7BB480067A98
:100B80000B7BC88000E564D5E001227902E453F2D2
:100B9000DFD5E0FDD29543F220D5E0FD53F2DFD55D
:100BA000E0FDC29543F220D5E0FDE920E005D296B4
:100BB00043F24030E005D29443F210E564D5E0FD05
:100BC000E920E00353F2BF30E00353F2EF7496D50F
:100BD000E0FDD9B9EAF8D5E0FDD8FBDBA853F2DF98
:100BE0002253F28F53F28F75D5FF22788076FF085B
:100BF00076FF0876FF0876FF0876FF0876FF08760E
:100C0000090876FF087601788C76010876FF087669
:100C1000FF0876FF0876FF0876FF0876030876FF60
:100C20000876FF0876FF0876250876D0087628082B
:100C300076500876040876FF0876020876FF087674
:100C40007A0876FF0876070876010876FF0876FFAF
:100C500008760008760022FA75F00CA4ABF0EAC31F
:100C600033F8740133F9E8C333F8E933F9E8C32BF7
:100C7000F8E93400F9E8C333F8E933F9227888E673
:100C8000C39403D23A5002C23AC238E630E102D2EB
:100C900038A23892397886E6149000809378A6F6C8
:100CA0007886E6F53FC394025003753F02789CE6D0
:100CB000753EFFB40203753EA0B40303753E82780F
:100CC000A0E6F8600674282409D8FCF5697896E651
:100CD000915788318932789EE691578833893478E4
:100CE00097E691578835893671E1223036117A00BE
:100CF0007B007CFF7D007E00B1518B618A602230D9
:100D00003A227896E6FA7B00789EE6FC7D00C3EAFC
:100D100033FAEB33FBC3EC33FCED33FD7E0AB15108
:100D20008B638A627896303A02789EE6FA7B007886
:100D300097E6FC7D007E00303A10C3EA33FAEB33CD
:100D4000FBC3EC33FCED33FD7E0AB1518B618A604D
:100D500022C3EC9EFCED9400FDC3EC9AFCED9BFDE0
:100D6000C3EC9423ED940050047C237D00C3EC94E9
:100D7000FFED940140047CFF7D017BFF0B7A000AAC
:100D8000EA7009C3EC33FCED33FDA17CEC8AF0A4DE
:100D9000AEF0ED8AF0A42E947C40E4EAF460DD220B
:100DA000D23691EB1205A31205A37A007B007C10CA
:100DB00012059BE5542AFA74003BFBDCF37C04C368
:100DC000EB13FBEA13FADCF7FFEB60027FFFC2369E
:100DD00091EB2278A5E6F954037000E9540C7000F9
:100DE000E954307000E954C07000227567007568DE
:100DF000007597DE7597AD7581C043FF8075EF066E
:100E000075A90071E17580FF75F19375A400758077
:100E1000FF75D4FF75900075F28F75A57075900001
:100E200075D5FF75A60175E34075E20271E1E4F83E
:100E3000F6D8FD71EB12147E78988664753001C285
:100E4000AF1205AB716D1205A371731205A3717911
:100E50001205A3B1D3C2AF75670075680078FA793F
:100E6000FA308707D9FBD8F7021C00917D91EB7807
:100E700098866471E175A91375A71075C10075A7EF
:100E80000075660075E407758811758E047589090B
:100E900075C80475910475D84075D90875F78275C1
:100EA0009E0375960175DB4275DA4275A82375E6D7
:100EB0009075B801759B80759D0075D10C75BCB996
:100EC00075BB1075E88075B201120597D2AF753CFD
:100ED00000C2301205ABC231C232C233C2347552C5
:100EE000007553007522001205A7C3E522940A502D
:100EF00002E1BBD2317522001205A7C3E522940A94
:100F00005002E1BBC231D2327522001205A7C3E5FF
:100F100022940A5002E1BB75E4F7758851758E0181
:100F20007589AA758C00758D00C2A9D2ABD2AA753D
:100F30006B80756A14756E50C232D23475220A12F3
:100F400005A7756A10C3E522940A7552007553000F
:100F50004069758E0C756B00756A28756E28752250
:100F60000A1205A7756A20C3E522940A7552007516
:100F700053004047758E0C756B80756A14756E143E
:100F800075220A1205A7756A10C3E522940A7552E4
:100F900000755300402575E407758811758E04753A
:100FA0008909D2A9C2ABC2AAC234D23375220012B7
:100FB00005A7C3E522940A4002C15512059B2030C3
:100FC00003020E55C2AF716D716D716DD2AF120516
:100FD000AB203403303A0302108112059B788CE673
:100FE000C394015003021081E530C3940150030201
:100FF00010817567A57568F17F02D23691EB1205F5
:10100000A7C2AFC236120CEBC3E554947FD2AF40F7
:1010100070120597C2AF120B7FD2AFDFDD120DA0A9
:10102000C3EF7897F61205ABB16B7F0AD236120C7C
:10103000EB1205A7C2AFC236120CEBC3E554947F86
:10104000D2AF50E6120597C2AF120B6D12059F1278
:101050000B6DD2AFDFD6120DA0EF24037896F6F811
:101060007997E7C394234003985006E824237897A0
:10107000F61205AB91C5B19A1205A7120CEB020E40
:10108000557567007568001205A7C3E554940140C3
:1010900003020FD1C2AF120B7F120B7F120B7FD254
:1010A000AF1205AB753000E4F537F5380537E53795
:1010B000F4703F0538789AE6781914601278321483
:1010C000600D787D14600878FA146003753800C3E9
:1010D000E53898401D120BE1120597153875370059
:1010E00078998664C2AF120B7FD2AF78988664126B
:1010F00005A712059FE5237003020E55C3E554941E
:1011000001500AC3E552940150160210AC1205A713
:10111000E5237003020E557552007553000212C28A
:10112000C3E55294017017C2AF120BE1789986643F
:10113000120B6D78988664D2AF1205A741B4C3E54F
:101140005294027017C2AF120BE178998664120BA9
:101150007378988664D2AF1205A741B4C3E5529460
:10116000037017C2AF120BE178998664120B79787D
:10117000988664D2AF1205A741B4C3E552940470B7
:1011800017C2AF120BE178998664120B7F789886AC
:1011900064D2AF1205A741B4C3E55294057017C2DB
:1011A000AF120BE178998664120B7F78988664D22F
:1011B000AF1205A741B4C3E55294077019C3E553B4
:1011C0009406500201FC7401303A0274037888F6E8
:1011D000C238C23941B4C3E55294087019C3E5530B
:1011E0009406500201FC7402303A0274047888F6C6
:1011F000D238D23941B4C3E55294097017C3E553CC
:101200009406500201FC303A0BC37888E69402F64B
:10121000C23A41B4C3E552940A7016C3E55394062A
:10122000500201FC203A0A7888E62402F6D23A41BC
:10123000B4C3E55294147025C3E5539406500201DB
:10124000FCC2AF901A0B740093D2AF7888F613C229
:1012500038C2394002D2384002D2398057C3E552F1
:1012600094157038C3E5539406404FC2AF901A0BE3
:10127000740093D2AFF8B801027402B8020274018C
:10128000B803027404B8040274037888F613C238F1
:10129000C2394002D2384002D2398018C3E5529494
:1012A0000C70117567A57568F1C3E5539406400A83
:1012B00091C5D2AF7552007553007567007568000F
:1012C00001FCC2AF120BE1E4D2AFE4F55EF524F508
:1012D00025F53D755E0812059712060030EDFDA854
:1012E000BDA9BEE97001F8885F120604755E08C2E8
:1012F000AF12066B855D5B855D5CD2AF75A710751F
:10130000C13075A70075A903756601303A07C23868
:10131000303502D238D228753900120B0C120B3D31
:1013200012067A12068112067A12068112067A12C3
:101330000906120A03120A481206811208F6202C26
:10134000031205BA302C031205EA120A03120A79B5
:10135000120681120906120A03120AAA1206811243
:1013600008F6120A03120ADB120681120906120A93
:1013700003120B0C1206811206001208F6120A0361
:10138000120B3D120604120681302827855D5B7919
:10139000187A0CC3E53999400EC228D2298A3B85B8
:1013A0005D5B855D5C800CC3E554940140030213D2
:1013B0002F813930291F202B1CE53B147006C229D0
:1013C000D22A612FF53B203A07C3E554940140032C
:1013D00002132F8064753C00203A0F78FA79A4E755
:1013E00060027803C3E55598504FE523604B303ACF
:1013F00017203805203507800F303502800A202B52
:1014000007D22B855D5B615F78F0302B05855D5BD6
:101410007820C3E54898500302132F302B1BC22BB2
:10142000C238303502D238D229753B12855D5B61F6
:101430002F053CE5546002813C753C00C2AF120BA5
:10144000E175240075250075A91375A71075C100F5
:1014500075A700756600D2AF1205A7120BE178A43C
:10146000E6600FC29643F240C29543F220C2944315
:10147000F210C3E53C94044003020E5501A7901AF4
:101480000D782091FEE520B4550AA391FEE520B425
:10149000AA0280137567A57568F1120BEB91C575EB
:1014A0006700756800801D901A0378807B0A91FEA2
:1014B000A308DBFA901A0F788C7B1A91FEA308DB45
:1014C000FA901A2922C2AFB141B11E901A007410CD
:1014D000B103A37407B103A37421B103901A037875
:1014E000807B0AB102A308DBFA901A0F788C7B1A72
:1014F000B102A308DBFAB154B132901A2922E49365
:10150000F622E6438F01538FFDFFC3E583941C4011
:101510000122EF8567B78568B7F0538FFE22438FAE
:1015200002438F018567B78568B7901A0DF0538F16
:10153000FC22901A0D7455B103901A0E74AAB103CF
:10154000227A3079D07820901A4091FEE520F70970
:10155000A3DAF7227A3079D0901A40E7B10309A3D1
:10156000DAF9227C051205ABDCFB22C2AF120B6D4F
:10157000120B73120B79120B7F12059F120B6D1257
:101580000B73120B79120B7F12059F120B6D120B4E
:1015900073120B79120B7FD2AF22C2AF120B7F12E4
:1015A0000B79120B73120B6D12059F120B7F120B2E
:1015B00079120B73120B6D12059F120B7F120B79B0
:0915C000120B73120B6DD2AF2265
:1019FD00020DEB100721FFFFFFFFFFFF09FF01FFA6
:101A0D0055AA01FFFFFFFFFF03FFFFFF25D0285061
:0D1A1D0004FF02FF7AFF0701FFFF0000FF3A
:101A400023575F485F31352320202020202020208D
:101A500023424C48454C492445464D3842323123B7
:101A60002020202020202020202020202020202076
:101C0000C2AFC2D37597DE7597AD7581C075A90057
:101C100043FF80752438752503B1DB7529A5752A26
:101C2000F143F18053A47FD28775D4FF75E3407DE3
:101C3000FA780379E67C10752200752300901DE880
:101C40007B06752498752501308702814820870816
:101C5000D8FBD9F9DCF781BA308708D8FBD9F9DC91
:101C6000F781BAB19BE493A3C39A6004DDC381BA40
:101C7000DBDBB18D600281317B08E493FAA3B16EA6
:101C8000DBF87A30B16E752200752300B18DEAFC65
:101C9000EBFDC3ED94FE400EB18D8A278B28ED300D
:101CA000E0048A828B83B18D7AC270D8C3ED94FE32
:101CB000601950CEBD0029EC600F7520007521FF22
:101CC000752900752A000200008100A827A92808AC
:101CD00009D804D90281DDB191EAF281D10D81A642
:101CE000C3ED94035051EDA2E092007AC5C3E582A2
:101CF0009400E583941C508C200010438F02438F86
:101D0000018529B7852AB7F0300027A827A9280818
:101D100009438F01538FFDD804D902A132C3E58353
:101D2000941C4003A3A117E28529B7852AB7F0A325
:101D3000A117538FFC81827AC1BD030CE493A3FAEF
:101D4000B152DCF8B14A81828184AA22AB23B16E00
:101D5000EBFAEA6222752608C3E52313F523E52290
:101D600013F52250066323A0632201D526EAB1DBD6
:101D7000B1DB75260AEAF4200102D287300102C2E3
:101D800087B1DBC3134002C201D526EB22B191EA31
:101D9000FB208702A191308702A196752608AE2408
:101DA000AF25C3EF13FFEE13FEB1DFB1DBC3EA13C0
:101DB0003087024480FA30E703632201C3E523132E
:101DC000F523E52213F52250066323A0632201D5F3
:101DD00026D9E52265236523F52222AE24AF250E00
:101DE0000FDEFEDFFCD20122424C48656C693437BD
:061DF0003164E8B20601B7
:00000001FF
